:020000020000FC
:100000000C9456000C948F0B0C948F0B0C948F0B4C
:100010000C948F0B0C948F0B0C948F0B0C948F0BF8
:100020000C948F0B0C948F0B0C9414000C941600F2
:100030000C948F0B0C948F0B0C948F0B0C948F0BD8
:100040000C948F0B0C948F0B0C948F0B0C948F0BC8
:100050000C948F0B0C948F0B0C948F0B0C948F0BB8
:100060000C948F0B0C948F0B0C948F0B0C948F0BA8
:100070000C948F0B0C948F0B0C948F0B0C948F0B98
:100080000C948F0B0C948F0B0C948F0B0C948F0B88
:100090000C948F0B0C948F0B0C94BF0A0C948F0B49
:1000A0000C948F0B0C948F0B0C948F0B0FEF0DBFD8
:1000B0000AE00EBF46D57894C2D16FEF91D1DDD161
:1000C000FACFE395C8953196002009F0089500E035
:1000D0000093B90567C5E0E2F7E1F4DF091679F4AA
:1000E000F1DF081669F4EEDF071659F43196C8956A
:1000F000002D3196C895F02DE02F09950895319681
:1001000031963396EACF90EF80EF21E008813CD121
:10011000513011F41AD0F7CF702F17D00D3091F065
:10012000352E088131D10D3069F0351639F4982F0C
:10013000872F702F0AD02395233099F7088124D177
:10014000351609F0089501D0F9CFDD1539F4CC1535
:1001500029F404E00093B90525C508952197089571
:1001600020E25ED120E25CD120E25AD120E258D1D7
:10017000392F4FD120E254D1382F4BD120E250D12A
:10018000372F47D120E24CD1089520E249D120E217
:1001900047D13E2F3ED120E243D108950BE000939A
:1001A000B90500C5D5E0CFE3552444247727BF7DAA
:1001B0000881CA9543940D3041F0E6D0523039F0B1
:1001C000B0625130A9F35394F3CF052D0895B5FFD4
:1001D0007395EECF04E00093B905E4C402E0009308
:1001E000B905E0C49F708F707F70EDD10895D5E0A0
:1001F000CFE3E03099F308810083319721970D30E8
:10020000C1F7AE2EBF2E0895CDDF743038F60B2D1A
:10021000043021F40A2D043F09F452C0D5E0CFE3A5
:10022000772788279927CC15AAF20881ADD05230BC
:1002300029F4982F872F702F2197F5CFD3DF672EC2
:10024000FB2DEA2DB77FBF7E992788277727772454
:100250003196F43011F4E53F59F0008195D05430D7
:1002600039F0523089F77394782F892F902FF0CF7F
:10027000072D033029F07394782F892F90E0F8CF61
:10028000B4FD02C0B061E0CFADDF671699F118F49C
:10029000B8609F2E8E2EF43021F4E53F11F4B3FFA9
:1002A0000FC0B3FF08C0761508F443C0F43019F44A
:1002B000E53F09F43EC0F43039F6E53F29F60895EC
:1002C00071DF003009F40895D5E0CFE3FB2DEA2D6E
:1002D000F13019F4E03009F409C008810083319746
:1002E00021970D30A9F7AE2EBF2E089502E000939E
:1002F000B90558C43197DF2FCE2FD13019F4C03053
:1003000009F468CF088121970D30B9F70E2F0C1B27
:10031000A00E08F4B394D13011F4C03029F0088154
:10032000008321973197F7CF3DDF003009F06CCF84
:10033000089538DF003039F10B2D013021F40A2DFA
:100340000050041598F2FB2DEA2DDF2FCE2FC41993
:10035000D0400C2FA02E0D2FB02EF91519F4E81552
:1003600009F405C00081088321963196F6CFD5E0C7
:10037000CFE3F92DE82D3197088100830D3019F076
:1003800031972197F9CF08955527102F1D3009F483
:1003900016C01F75103009F402C01C3011F451E072
:1003A000089510310AF408951B350AF008951034A9
:1003B00012F053E008951A310AF452E0089554E01F
:1003C0000895CF3319F427E02BD00EC028E03CD09D
:1003D00020E23AD0212F38D0C3951DE0188304C005
:1003E0002EE31ED0D5E0CFE334D0183051F31F37C1
:1003F00041F31A3009F4F8CF18831D3049F0C030AA
:1004000019F427E00DD0F0CFCA95212F1DD0ECCFE5
:100410000895BED0242F04D0232F02D00895202F7A
:100420000090C80005FEFCCF75D3B6FF05C0009054
:10043000C80007FEFCCFBF7B2093CE0008952DE0BF
:10044000EFDF2AE0EDDF08952D3011F4F8DF089595
:10045000E7CF889500000091C80007FFFACF109100
:10046000CE000895C895002021F0202DD9DF3196C7
:10047000F9CF0895F7DFE3DF0895D5E0CFE30FEF7D
:10048000C02E05E0D02E08817FDF523009F4BCCEAB
:10049000D6DFA16001C0AE7F3DB73F3C20F408E04D
:1004A0000093B9057FC32FDE7D30C9F07B33B9F0EF
:1004B000032D023031F49F708F707F7084D022D072
:1004C000EBCF9F758F757F75213029F4032D033095
:1004D00011F407D0E1CFFFDD7D3009F00895A16070
:1004E000089571547A3122F005E00093B9055AC39A
:1004F000705CA0FF11F406D00895F5E0E72F70813D
:1005000001D00895F4E0E62F70836A95633F20F4EC
:1005100006E00093B90546C308956395603022F064
:1005200007E00093B9053EC3F4E0E62F708108951B
:10053000F4DF07E007174AF001E0703019F0000F10
:100540007A95FBCF702FDEDF08950AE00093B9059E
:1005500029D3903039F0905D292F62DF803011F47B
:1005600020E35EDF803019F0805D282F59DF705D59
:10057000272F56DF089599278827745610F09395F2
:10058000FCCF7C597A5010F08395FCCF765F0895AC
:10059000432F4695469546954695405D4A3308F06B
:1005A000495F3F70305D3A3308F0395F089546FD8A
:1005B000475F4F7036FD375F3F70440F440F440F65
:1005C000440F342B08959330B2F4923032F08630D9
:1005D00092F4853012F0763072F4882321F00AE02C
:1005E000700F8A9581F7992309F4089504E6889499
:1005F000700F9A95C0F701E00093B905D3C2E2E607
:10060000FAE138DF08951BDFF4E0E4EFFB1511F4A5
:10061000EA1521F0208118DF3197F8CF10DF0FDFC6
:10062000E2E7FDE11FDF7A2D9B2D705091406ADFDC
:10063000792FA1DF8EDFE0E8FDE114DF6EDF9BDFC5
:1006400088DFFDDE0895AE7F27DF67DF94DF81DF7F
:10065000F6DE089520DF24E2E3DE5FDF372FD9DE08
:10066000EEDE0895AE7F18DF58DF072F56DFF5E086
:10067000E72F00830895A2FF72C0AE7F0DDF4DDF2C
:10068000672E4BDF872F49DF772EF5E0E72F80833A
:10069000A062A860AA7F0895F5E0E72D0081061505
:1006A00019F003950083A0610895F5DE36DF072F6A
:1006B00034DF701719F0772725DF08957FEF22DFE9
:1006C0000895E9DE70E000B605FE71E01BDF0895D5
:1006D000E2DE23DFE72FF0E0708114DF0895DBDE38
:1006E0001CDF072F1ADFF0E0E02F70830895D3DEC0
:1006F00014DF072F12DF709F1120F09B19F4702D6B
:1007000001DF08950FE00093B9054CD2C4DE05DF88
:100710007723F09B99F0072F00DF872F991B79E053
:10072000881F7A9541F0991F901B18F4900F8894B8
:10073000F7CF0894F5CF782FE5DE089501E1009317
:10074000B90530D2A8DEE9DE072FE7DE700FF09B97
:1007500010F0D8DE08950FE00093B90523D29BDE98
:10076000DCDE072FDADE701BF09B13F0CBDE089582
:1007700000E10093B90516D28EDECFDE072FCDDE65
:100780007023C0DE089587DEC8DE7695BBDE08954F
:1007900082DEC3DE770FB6DE08957DDEBEDE072F74
:1007A000BCDE702BAFDE089576DEB7DE072FB5DE38
:1007B0007027A8DE08956FDEB0DE7095A3DE089581
:1007C0006ADEABDE71959EDE089571E09BDE0895D2
:1007D00062DEA3DE072FA1DE701705C05CDE9DDEA2
:1007E000072F9BDE071770E082F779F38BDE089501
:1007F00052DE93DE772309F0A26008950DB70E5FF5
:100800000DBF0895A460089546DE0895B26008956E
:1008100048819BDC3881CBDE732F74DE96DC3BDEB7
:10082000089539DE7ADECF93DF93D0EAC9EFCA9517
:100830000000E9F7DA950000C9F77A95B1F7DF9182
:10084000CF91089577275EDE26DE67DE01E0071789
:100850002AF0F09870FD01C0F09A08950CE0009322
:10086000B905A0D118DE59DE472FF4E0E4EF0AC045
:10087000FB1511F4AE16E8F400810D3011F031973C
:10088000F7CF3197772788279927FB1511F4AE16F4
:1008900080F4008179DD523029F4982F872F702F52
:1008A0003197F3CF9F708F707F708DDE471701F700
:1008B000089509E00093B90575C1D4DFDF2FCE2F6D
:1008C0000895D0DFA06C0895B2FF02C0B160089512
:1008D000B2600895E0DD21DE272FA2DD089588951E
:1008E00000000091C80007FFFACF7091CE0073306E
:1008F00009F4B26007DE0895CEDD0FDE08E020E3E4
:10090000771F08F421E38CDD0A95C9F798DD089577
:1009100004EB7091BA05779508F470277093BA05C7
:10092000F1DD0895427265616B200A0D0000D4E08C
:10093000C4EF6FEFA160EED0A5FF03C08C2E9D2EFB
:10094000AF7DA4FF03C0D92DC82DAF7EA6FF03C085
:100950004C2E5D2EAF7BA7FF04C0DF2FCE2FB460DF
:10096000AF77B0FF03C0D52DC42DBA7FB1FF04C04F
:10097000CDD0DB2DCA2DBD7FDB1511F4AC1678F47C
:10098000088102DDA1FF04C0543011F02197D1CFBE
:10099000AD7F523011F42197CCCF7EDDCACF0895C0
:1009A00004E0B02E04EFA02EFB2DEA2D6FEFA0E0A7
:1009B000B0E0F1E0E0E000E00193F430E8F3E43F80
:1009C000D9F7F5E0E0E400E00193F530E8F3EA352B
:1009D000D9F735DDEAEDF9E14DDD0895EEE5FCE10D
:1009E00041DDEAE3FDE13EDD08E1202EF4E0E4EF45
:1009F0003F2F0FDD3E2F0DDD2AE312DD20E210DD5B
:100A0000F13011F4E03099F0308103DD20E208DDAF
:100A100031972A9459F413DD3F2FFBDC3E2FF9DC8C
:100A20002AE3FEDC20E2FCDC08E1202EE9CF07DD32
:100A300006DDE6E5FDE116DD3B2DEBDC3A2DE9DCDC
:100A4000FEDCEEE5FCE10EDDFADC0895EEE5FCE10E
:100A500009DDE6ECFCE106DD08E1202EF3E0EFEF36
:100A60003F2FD7DC3E2FD5DC2AE3DADC20E2D8DCCE
:100A70000F93E03000E0F0070F91B1F0F2BDE1BD5F
:100A8000F89A30B5C6DC20E2CBDC31972A9459F4D1
:100A9000D6DC3F2FBEDC3E2FBCDC2AE3C1DC20E2EB
:100AA000BFDC08E1202EE4CFCADCEEE5FCE1DADCB5
:100AB000C6DC0895EEE5FCE1D5DCE0EBFCE1D2DC40
:100AC00008E1202EE0E4F5E03F2FA3DC3E2FA1DC7F
:100AD0002AE3A6DC20E2A4DCEA3591F0319199DC2E
:100AE00020E29EDC2A9459F4AADC3F2F92DC3E2FB0
:100AF00090DC2AE395DC20E293DC08E1202EECCFA9
:100B00009EDCEEE5FCE1AEDC9ADC0895E4E2F9E07F
:100B1000A9DC08950090C80007FE0BC00091CE002C
:100B2000033111F4B06405C00091CE00033009F424
:100B3000B2600895DF93D4E0DA950000E9F7DF9121
:100B4000089506E204B900E005B900E007B900E045
:100B500008B908E00AB900E00BB900E00DB900E0FF
:100B60000EB900E000BB00E001BB00270093BB050D
:100B70000EBB74EB0091000107270093BA0500E05B
:100B80000093CD0003E30093CC0008E90093C90073
:100B900001E003BF0E94D004489902C046D4C7DEDA
:100BA0002EDD08954CDC0091B905E9EDF5E0E00F8C
:100BB000099415C017C019C01BC01DC01FC021C09B
:100BC00023C025C027C029C02BC02DC02FC031C0D5
:100BD00033C035C037C039C03BC03DC03FC0EAE874
:100BE000FDE13FD0E2EBFDE13CD0E0EFFDE139D0AB
:100BF000E2E1FEE136D0E4E5FEE133D0E4E8FEE1F7
:100C000030D0E8EBFEE12DD0EAEFFEE12AD0EAE5B4
:100C1000FFE127D0EAEBFFE124D0E2EFFFE121D0B2
:100C2000EAE2F0E21ED0EEE5F0E21BD0E6E9F0E207
:100C300018D0EEECF0E215D0E8EFF0E212D0E6E1E9
:100C4000F1E20FD0E6E3F1E20CD0E0E5F1E209D009
:100C5000E2E7F1E206D0E8E9F1E203D0EEEBF1E2FF
:100C600000D000DC0FEF0DBF0AE00EBF0FEF0DBF8D
:100C70006FEFA0E0B0E0E3DB1ECA772743DC0BDCBC
:100C80004CDC01E00717A2F00CE070FD08E40093D3
:100C9000B800409A419A00270093B900009500934C
:100CA000BB0004E00093BC0004E90093BC0008957D
:100CB0000CE00093B90576DF0091BC0002FF25C06F
:100CC000EADB2BDC7093BB0005E80093BC000091CD
:100CD000BC0007FFFCCF0091B900087F083111F07C
:100CE000003439F47091B9007695769576950ADCE2
:100CF0000895003231F0083421F002E10093B90583
:100D000051DF04E10093B9054DDF03E10093B9051C
:100D100049DF0091BC0002FF21C0BDDBFEDB709308
:100D2000BB0005E80093BC000091BC0007FFFCCFAE
:100D30000091B900087F083239F47091B9007695B6
:100D400076957695DFDB0895003321F002E100937C
:100D5000B90528DF04E10093B90524DF03E100931E
:100D6000B90520DF0091BC0002FF23C071E0CADB9F
:100D700092DBD3DB01E0071702F104EC70FF04E81B
:100D80000093BC000091BC0007FFFCCF0091B900AC
:100D9000087F003521F47091BB00B4DB0895003565
:100DA00021F002E10093B905FDDE04E10093B905ED
:100DB000F9DE03E10093B905F5DE0CE00093B90517
:100DC000F1DE0091BC0002FF11C004EA0093BC00F8
:100DD0000091BC0007FFFCCF0091B900087F0830EC
:100DE00009F4089502E10093B905DCDE03E1009304
:100DF000B905D8DE0091BC0002FF0BC004E90093E6
:100E0000BC000FEF0093BB00089502E10093B90509
:100E1000C9DE03E10093B905C5DE0091BC0002FF05
:100E200011C00091BC0004FF02C070E809C000912D
:100E3000BC0007FFFCCF7091B9007695769576954A
:100E400061DB089503E10093B905ACDE72E05ADB83
:100E500022DB63DB03E0071742F0770F770F51D0F7
:100E60000CB5037F072B0CBD08950DE00093B90569
:100E700099DE11DB52DB01E007174AF00CB5006286
:100E80000CBD70FD03C00CB50F7D0CBD08950CE0CA
:100E90000093B90587DEFFDA40DB07E007177AF039
:100EA000072E73700CB5087F072B0CBD0DB50160C4
:100EB0000DBD02FC03C00DB50E7F0DBD08950AE007
:100EC0000093B9056FDEE7DA28DB28980000000000
:100ED0007EBD0DB407FEFDCF7EB5089528980000B5
:100EE00000007EBD0DB407FEFDCF7EB50BDB08957F
:100EF00071E008DBD0DA11DB289A70FD01C0289878
:100F0000089504B1076004B905B1016005B901E5B0
:100F10000CBD0DB50E7F0DBD0895009164000E7FD0
:100F20000093640000E000937B007727EBDAB3DAEC
:100F3000F4DA00917C00007E80917B008F7D8093AD
:100F40007B0076FF04C080917B00806280937B00F1
:100F50007F71072B00937C0007EC00937A000091CF
:100F60007A0006FDFCCF07EC00937A0000917A002E
:100F700006FDFCCF70917900C5DA08957727C2DAB3
:100F80008ADACBDA01E0071752F000917C000F7388
:100F9000006270FD01C0006C00937C0008950CE0BD
:100FA0000093B905FFDD74B1ADDA089574DAC0DAE3
:100FB000B4DA05B1072B05B908956DDAB9DAADDAFF
:100FC000709505B1072305B9089565DAB1DAA5DA98
:100FD00004B1072B04B908955EDAAADA9EDA709597
:100FE00004B1072304B9089556DAA2DA96DA03B1F8
:100FF000072370E0002309F471E084DA08954BDAE6
:101000008CDA75B9089547DA88DA74B9089573B13E
:1010100079DA089577B176DA08953DDA89DA7DDAFA
:1010200008B1072B08B9089536DA82DA76DA7095B6
:1010300008B1072308B908952EDA7ADA6EDA07B113
:10104000072B07B9089527DA73DA67DA709507B1C5
:10105000072307B908951FDA6BDA5FDA06B10723B1
:1010600070E0002309F471E04DDA089514DA55DADE
:1010700078B9089510DA51DA77B9089576B142DA7D
:1010800008957AB13FDA089506DA47DA7AB9089511
:1010900002DA4EDA42DA0BB1072B0BB90895FBD90D
:1010A00047DA3BDA70950BB107230BB90895F3D9F2
:1010B0003FDA33DA0AB1072B0AB90895ECD938DAE6
:1010C0002CDA70950AB107230AB90895E4D930DA09
:1010D00024DA09B1072370E0002309F471E012DA81
:1010E0000895D9D91ADA7BB9089579B10BDA089540
:1010F0007DB108DA0895CFD910DA7DB90895CBD93A
:1011000017DA0BDA0EB1072B0EB90895C4D910DA2D
:1011100004DA70950EB107230EB90895BCD908DA28
:10112000FCD90DB1072B0DB90895B5D901DAF5D960
:1011300070950DB107230DB90895ADD9F9D9EDD941
:101140000CB1072370E0002309F471E0DBD90895A6
:10115000A2D9E3D97EB908957CB1D4D9089570B3EA
:10116000D1D9089598D9D9D970BB089594D9E0D927
:10117000D4D901B3072B01BB08958DD9D9D9CDD9C5
:10118000709501B3072301BB089585D9D1D9C5D97D
:1011900000B3072B00BB08957ED9CAD9BED970957C
:1011A00000B3072300BB089576D9C2D9B6D90FB1D1
:1011B000072370E0002309F471E0A4D908956BD9E6
:1011C000ACD971BB08957FB19DD9089564D901E868
:1011D0000093800009E000938100002700938200C3
:1011E000259A9BD900270093890070938800089561
:1011F00052D903E80093800009E0009381000027A2
:1012000000938200259A89D9072F87D97093890086
:1012100000938800089500270093800008957727A1
:1012200071D939D97AD907E0071772F00091BB0557
:10123000087F702B7093BB050027009382000093FA
:1012400080000093810008950AE00093B905AADCAC
:1012500071E058D920D961D901E007174AF000910F
:10126000BB050F7770FF01C000680093BB050895B0
:101270000CE00093B90596DCCF93DF93882777279E
:1012800076BB8093850070938400B09A0091BB0573
:10129000902F9078C894991F991F96600770E3E586
:1012A000F9E0E00F09947AC006C005C004C02AC066
:1012B00029C028C04FC0033008F005E0909381009A
:1012C0008093850070938400D0E1C3EFCA9500003D
:1012D000000000000000D1F7CFEFCA950000000029
:1012E0000000D9F7CCEFCA95000000000000000014
:1012F000D1F716F06894E9CFDA95E89431F70A95BA
:1013000019F74CC00350033008F005E090938100BA
:101310008093850070938400D0EAC3EFCA950000E3
:10132000000000000000D1F7CFEFCA9500000000D8
:101330000000D9F7CCEFCA950000000000000000C3
:10134000D1F716F06894E9CFDA95E89431F70A9569
:1013500019F724C0909381008093850070938400D6
:101360000AE0D0EAC3EFCA950000000000000000C8
:10137000D1F7CFEFCA95000000000000D9F7CCEFFD
:10138000CA950000000000000000D1F716F0689434
:10139000E9CFDA95E89431F70A9519F7709184004E
:1013A00080918500002700938100B09908C0C9E5AD
:1013B000D5E088830E948202DF91CF910895DF916A
:1013C000CF910EE00093B905EDDBD4E0CFEFF5014E
:1013D000CE1BDF0BF3E0EFEFEC17FD0724F4E8ED95
:1013E000FCE148D80895EEEFFCE144D86FEF7A2D88
:1013F00089D87B2D87D8D4E0CFEFF3E0EFEF0881D9
:10140000F999FECFF2BDE1BD00BDFA9AF99AD1304B
:1014100011F4C03049F031970F93E03000E0F0074D
:101420000F9111F02197EBCF0895E6E2FDE122D86C
:10143000B7DAD4E0CFEFEFEFF3E0F999FECFF2BDEA
:10144000E1BDF89A00B50883D13011F4C03019F02D
:1014500031972197F2CF6DEF60D8B72EF72F5DD877
:10146000A72EE72F0F93EF3F04E0F0070F9131F421
:10147000E0E1FDE10E943A020E94D00408950BD8F9
:101480004CD8172F88940BD0089505D846D8172F1D
:10149000089405D0089527D0712F34D808950AB143
:1014A000077E0AB90BB108610BB999E04B9BFECFDF
:1014B0005C9A549810F05C98549A5B98539A2FD089
:1014C00053985B9A2CD04B99F8CF18F05C9A5498AB
:1014D00002C05C98549A4B9BFECF54985C9A111FA3
:1014E0009A9521F708950AB1077E0AB90BB10861F0
:1014F0000BB999E04B99FECF88944C9B06C0089499
:101500005B98539A4C99FECF04C05B98539A4C9BBE
:10151000FECF53985B9A111F9A9561F7089530E5B5
:1015200040E54A95F1F73A95D9F70895CF93DF93BF
:1015300077270E9482020E944B020E948D020717A9
:10154000D2F070FD0BC0CDD0CFEBD5E0099309935D
:1015500008835C9A5498DF91CF910895C7E5D5E050
:1015600039D000270093C205549A5C9894D0DF913B
:10157000CF91789408950CE00093B90513DB9F9305
:101580009FB79F938F937F93EF93FF93FEE7E09135
:10159000C2057091BF058091C0059091C105E70E0D
:1015A000F81EE91F7491E093C20570FF0AC00000A5
:1015B0005C9AFF91EF917F918F919F919FBF9F9137
:1015C00018955C98FF91EF917F918F919F919FBFAC
:1015D0009F911895C7E5D5E03327442755279927CC
:1015E0008827772700EF102E088001200294002022
:1015F00041F030E0731F40E0841F50E0951F0A94D3
:10160000F6CF099012940120002041F039E9731FB0
:1016100049E9841F59E1951F0A94F6CF0880129476
:1016200001200294002041F03CE5731F4FE8841F25
:1016300052E0951F0A94F6CF0990129401200020E1
:1016400041F039E8731F41E4841F50E0951F0A946C
:10165000F6CF0880129401200294002041F03DE86A
:10166000731F46E0841F50E0951F0A94F6CF088050
:1016700012940120002041F037EA731F40E0841FDC
:1016800050E0951F0A94B1F77093BF058093C00591
:101690009093C1050895009165000F7E0093650049
:1016A000002709BB0093BE000093C0000093C10057
:1016B0000093CF000093D0000093C2000093C300BA
:1016C0000093C4000FE90093D10000E00093800074
:1016D00001E00093C1000091720000640093720069
:1016E0000895F894002709BB0093C0000093C1003F
:1016F0000093BE000093D0000093CF000093C2007F
:101700000093C3000093C400009172000F7B00930C
:1017100072000091650000610093650008951895BE
:101720004C495320030353495A200F034E45572079
:10173000D00450500B20A20350500D20AF03505046
:101740000A20770350500F208603414F5620220471
:101750005052494E2303505258202A0350524220DF
:101760007C04454D49546A04501A1D2032035050E0
:101770001D203B03464F522002044E4558544C0353
:10178000501C1E20550350501E20EE0350501C20AC
:10179000E80350494620F80350544F2004045050A9
:1017A0000420080452554E209704454E4420060458
:1017B000414E4420BC034C535220C3034C534C2095
:1017C000C803504F5220CD03584F5220D403434FEB
:1017D0004D20DB034E454720E003524E4420880451
:1017E00044454C411104474F544F5D04474F5355F6
:1017F00061045245545564045448454EFE034B451C
:1018000059206F0441434F20610353415645E50978
:101810004C4F4144150A5045454B6803504F4B45CA
:101820006F034F444220030849444220D3075344E6
:101830004220E50743444220EC074F504220FF0777
:1018400053424220D60743424220DD07494E422000
:10185000070849424220F4074F4443203A084944CC
:1018600043200A08534443201C08434443202308D0
:101870004F5043203608534243200D084342432033
:101880001408494E43203E08494243202B084F4448
:101890004420440849444420410853444420570804
:1018A000434444205E084F50442071085342442072
:1018B0004808434244204F08494E44207508494295
:1018C000442066084F4445200308494445207808D1
:1018D000534445208E084344452095084F504520E9
:1018E000A808534245207F08434245208608494EB8
:1018F0004520AC08494245209D084F444620B20887
:1019000049444620AF0853444620C5084344462076
:10191000CC084F504620DF0853424620B6084342C9
:101920004620BD08494E4620E30849424620D408D7
:1019300044554D50EE044544554D26055644554DED
:101940005A05445352454B0A4453434F450A4453A6
:1019500044453F0A494347200F0949434520280988
:10196000494350203C0950574D38E6085057452010
:10197000F80850574F200B0944445320960A41441D
:1019800043208D0741445220BE0753504D20260767
:1019900053504F203907535043204B075350572083
:1019A0006307535052206E07535053207807545703
:1019B00049203D0654575320E10654575020FA065B
:1019C000545741205C0654575720890654575220DB
:1019D000B206545742200D0700003D3D3D3D3D3DC0
:1019E0003D3D3D3D3D3D3D3D3D3D3D3D3D3D3D3D27
:1019F0003D3D3D3D3D3D3D3D3D3D3D3D3D3D3D3D17
:101A00003D3D3D3D3D3D3D3D3D3D3D3D3D3D0A0D69
:101A100020202020202020202020202020202020C6
:101A20004174746F42415349432041546D6567616D
:101A3000333255340A0D2020202020202020202061
:101A4000202020204275696C6420636F64653A2011
:101A500032303131303532362E31383333000A0DE1
:101A600000002D2D2D2D2D2D2D2D2D2D2D2D2D2D00
:101A70002D2D2D2D2D2D2D2D2D2D2D2D2D2D2D2D96
:101A80002D2D2D2D2D2D2D2D2D2D2D2D2D2D2D2D86
:101A90002D2D2D2D2D2D0A0D2020202020204F72A0
:101AA0006967696E616C20636F6465202843293221
:101AB0003030322062792052696368617264204359
:101AC000617070656C730A0D2020687474703A2F11
:101AD0002F70726F6A656374732E63617070656CCA
:101AE000732E6F7267202070726F6A656374734023
:101AF00063617070656C732E6F7267200A0D2D2DF7
:101B00002D2D2D2D2D2D2D2D2D2D2D2D2D2D2D2D05
:101B10002D2D2D2D2D2D2D2D2D2D2D2D2D2D2D2DF5
:101B20002D2D2D2D2D2D2D2D2D2D2D2D2D2D2D2DE5
:101B30002D2D0A0D2020204D3136382F33325534CB
:101B400020706F72742C205457492C205350492C0C
:101B500020444453202620496E70757420436170E0
:101B6000747572650A0D20202020284329323031F7
:101B7000312062792053636F747420566974616CEC
:101B800065206B73765F70726A40626967666F6F1B
:101B9000742E636F6D200A0D2D2D2D2D2D2D2D2DC5
:101BA0002D2D2D2D2D2D2D2D2D2D2D2D2D2D2D2D65
:101BB0002D2D2D2D2D2D2D2D2D2D2D2D2D2D2D2D55
:101BC0002D2D2D2D2D2D2D2D2D2D2D2D0A0D2020A2
:101BD000202020416C6C2072696768747320616EEC
:101BE000642072656D6564696573206578707265DF
:101BF00073736C792072657365727665642E0A0D55
:101C000020202020202020202020202020204E6F57
:101C10007420666F7220636F6D6D65726369616CAD
:101C2000207573650A0D3D3D3D3D3D3D3D3D3D3DCE
:101C30003D3D3D3D3D3D3D3D3D3D3D3D3D3D3D3DD4
:101C40003D3D3D3D3D3D3D3D3D3D3D3D3D3D3D3DC4
:101C50003D3D3D3D3D3D3D3D3D3D0A0D00002D2DB1
:101C60002D2D2D2D2D2D2D2D2D2D2D2D2D2D2D2DA4
:101C70002D2D2D2D2D2D2D2D2D2D2D2D2D2D2D2D94
:101C80002D2D2D2D2D2D2D2D2D2D2D2D2D2D2D2D84
:101C90002D2D2D2D2D2D2D2D2D2D2D2D2D2D2D2D74
:101CA0002D2D2D2D2D2D2D2D2D2D2D200A0D00000E
:101CB0005661726961626C657320696E2052414D94
:101CC0003A0A0D00000045455020436F6E74656E62
:101CD00074733A0A0D0000004572726F723A205018
:101CE000726F6772616D20746F6F206C61726765CF
:101CF00020666F7220454550210A0D000000536197
:101D000076696E6720746F204545502E0A0D0000DD
:101D10004572726F723A2045455020657261736555
:101D200064210A0D00004C6F6164696E6720667261
:101D30006F6D204545500A0D000050524F475241EB
:101D40004D204D656D6F727920436F6E74656E74B2
:101D5000733A0A0D00004E65787420617661696CF3
:101D600061626C65206C6F636174696F6E3A20000C
:101D7000000046726565202070616765733A000057
:101D8000202063686172733A00004572726F72209E
:101D9000303A20556E6B6E6F776E20636F6D6D619C
:101DA0006E64206F72206F70657261746F722E2086
:101DB00000004572726F7220313A20456E636F7574
:101DC0006E746572656420612076616C756520743F
:101DD000686174206973206E6F7420626574776522
:101DE000656E203020616E64203235352E20000073
:101DF0004572726F7220323A2050726F6772616D55
:101E0000206D656D6F72792069732066756C6C2E1C
:101E100000004572726F7220333A20456E636F7511
:101E20006E746572656420612063686172616374B9
:101E300065722074686174206973206E6F7420610C
:101E4000207265636F676E697A6564207479706566
:101E50002E2000004572726F7220343A696E7465EC
:101E6000726E616C206572726F72202D20627566D1
:101E7000666572206C696D69742065786365656458
:101E8000656400004572726F7220353A20496E61B8
:101E90007070726F707269617465207661726961C9
:101EA000626C65206E616D6520656E636F756E7422
:101EB000657265642E0000004572726F7220363ABA
:101EC000204461746120737461636B207075736862
:101ED000206572726F72202D746F6F206D616E7944
:101EE00020617267756D656E7473206F6E206F6E02
:101EF00065206C696E652E0000004572726F72205D
:101F0000373A204461746120737461636B20706F91
:101F100070206572726F722E0A0D20202020202002
:101F200020202046756E6374696F6E207472696537
:101F30006420746F2075736520612076616C75650F
:101F4000207468617420776173206E6F74206176ED
:101F500061696C61626C652E00004572726F72205F
:101F6000383A204D616368696E6520737461636BF4
:101F7000206572726F720A0D202020202020202000
:101F80002046756E6374696F6E7320616E642F6F87
:101F9000722063616C6C73206E6573746564207469
:101FA0006F6F20646565706C79206F7220746F6F3D
:101FB00020636F6D706C657800004572726F7220DF
:101FC000393A20474F544F206F7220474F535542A4
:101FD0002064657374696E6174696F6E206C696EDC
:101FE0006520776173206E6F7420666F756E642E46
:101FF00000004572726F7220413A20537065636928
:10200000666965642062697420706F736974696FB2
:102010006E2072616E6765206F6620303A372065EA
:10202000786365656465640000004572726F7220B4
:10203000423A204C696E65206E756D62657220684B
:102040006173206D6F7265207468616E20746872B0
:102050006565206E756D6572616C73200000457258
:10206000726F7220433A20537065636966696564D4
:102070002062697420706F736974696F6E20726179
:102080006E6765206F6620303A312065786365653C
:102090006465640000004572726F7220443A2053F8
:1020A00070656369666965642062697420706F7326
:1020B0006974696F6E2072616E6765206F6620308B
:1020C0003A33206578636565646564000000457295
:1020D000726F7220453A20496E70757420436170AA
:1020E00074757265207265676973746572206F76A6
:1020F0006572666C6F7700004572726F7220463AA7
:102100002041726974686D65746963206F766572C9
:10211000666C6F7700004572726F722031303A2022
:1021200041726974686D6574696320756E64657267
:10213000666C6F7700004572726F722031313A2001
:10214000446976696465206279207A65726F00005F
:102150004572726F722031323A20545749206275AD
:1021600073206572726F72206F63637572656400AD
:1021700000004572726F722031333A205457492063
:10218000696E74657266616365206E6F7420656E3A
:1021900061626C65640000004572726F72203134B8
:1021A0003A2054574920536C617665207265706CF3
:1021B0006965642077697468204E414B0000457260
:1021C000726F722031353A20756E75736564000048
:107E00000000000000000000000000000000000072
:107E10000000000000000000000000000000000062
:107E20000000000000000000000000000000000052
:107E30000000000000000000000000000000000042
:107E40000000000000000000000000000000000032
:107E50000000000000000000000000000000000022
:107E60000000000000000000000000000000000012
:107E70000000000000000000000000000000000002
:107E8000FFFFFFFFFFFFFFFFFFFFFFFFFFFFFFFF02
:107E9000FFFFFFFFFFFFFFFFFFFFFFFFFFFFFFFFF2
:107EA000FFFFFFFFFFFFFFFFFFFFFFFFFFFFFFFFE2
:107EB000FFFFFFFFFFFFFFFFFFFFFFFFFFFFFFFFD2
:107EC000FFFFFFFFFFFFFFFFFFFFFFFFFFFFFFFFC2
:107ED000FFFFFFFFFFFFFFFFFFFFFFFFFFFFFFFFB2
:107EE000FFFFFFFFFFFFFFFFFFFFFFFFFFFFFFFFA2
:107EF000FFFFFFFFFFFFFFFFFFFFFFFFFFFFFFFF92
:00000001FF
